:20C000002F4CC2935A023020829F560228281E4256020E8F3E9065002428D2435A02C29341
:20C020005B021420D2435B02924260025E021E425E021E825C020F433C4060EA0D43B0127F
:20C040003AC2824C540282436002053CC2435B02924260025C02924256025802023C824FCD
:20C06000560292536002123C1F9258020B281F8258023F9065000828C2435A0292425802A7
:20C080005602023C824F58029253600230410A1209127A4C213C1C530E930D243F900001BC
:20C0A0000A2C29434F4F8F107B4C0FDB1983FA23023C2F9202287B4C013C0B4A1F833F9341
:20C0C0000B244B4B1D53CD4BFFFF1F833F93FA23033C1D53CD4FFFFF7F4C0F9AFA237F4C5F
:20C0E0000F93E7237F4C8F106B4C0F5BD42330406EC30A1209123F40B4C33F90BAC31624BE
:20C100003F40BEC33F90C6C311243A40C6C33A80BEC30A110A113940BEC33C497F4C0F5F66
:20C120001F4FB4C33D498F121A83F7233F4000003F90000008243A400000023C3F4A8F12E0
:20C140003A900000FB2330406EC30A12091209430A431B430F930424094D0D4C0C430D3C17
:20C160000C5C0D6D0969098E04281CD30B5BF82B033C095E0B5BF42B1B430C5C0D6D096953
:20C180000A6A098E0A7F04281CD30B5BF62B043C095E0A6F0B5BF12B0E490F4A39413A4122
:20C1A00030410F120E120D120C120B12E2E229007F4028006F930C284E4F0E5E3E500002D0
:20C1C0004D4F0D5D9D4EFEFF00025F836F93F42F0C43B012B2C2824C00023C400002B012D3
:20C1E00000C0925352023B413C413D413E413F4100130A12B240805A2001B0127AC2B012F4
:20C200008CC3E2D22A0082435202B24010006201B24000026001B240E803720132D2B240D8
:20C2200010026001B01274C37C90480002205A4254020C4AB01280C3F53F0A120A430F9390
:20C2400005343EE33FE31E530F631AD30D9305343CE33DE31C530D633AE3B0124AC11AB3E4
:20C2600004243CE33DE31C530D632AB304243EE33FE31E530F633A413041C2435600D242F2
:20C28000FF105700D242FE105600F24006002600F24006004100F2D080006100F2406800AC
:20C2A0006200C2436300F2400A006400D2C3610030410D4CB2F0FF0FB001B012F8C282DC19
:20C2C000B2011C43B012E6C2C24C4A00B2D00300B001A2B2B001FD27A2C2B001C2434A00C7
:20C2E0001C42B40130413DF00F003DE00F000D5D005D0C5C0C5C0C5C0C5C0C5C0C5C0C5CB3
:20C300000C5C0C5C0C5C0C5C0C5C0C5C0C5C0C5C304131400004B012A0C30C930224B0124B
:20C32000F2C00C43B012F2C1B012A4C31F4C01000F9305241D53CD43FFFF1F83FB23304178
:20C340000F4C0C4D3D4003000D5F1E4F0100304052C30F4C0E9305241F53FF4DFFFF1E83C8
:20C36000FB2330413441354136413741384139413A413041D2B30300FD275C426600304154
:20C38000E2B30300FD27C24C67003041B2401010B001304132D01000FD3F1E4330408EC05A
:08C3A0001C4330410343FF3F41
:1EC3A80001010004010A0001000000002CC39AC340C300005600A8C35602BAC300027E
:02FFE00094C3C8
:02FFE40094C3C4
:02FFE60094C3C2
:02FFEA0094C3BE
:02FFEC0094C3BC
:02FFEE0094C3BA
:02FFF00094C3B8
:02FFF200A2C1AA
:02FFF40094C3B4
:02FFF60094C3B2
:02FFF80094C3B0
:02FFFA0094C3AE
:02FFFC0094C3AC
:02FFFE0012C32C
:00000001FF
